:03000000020040BB
:10004000C2B64396081203D812041D753B01120371
:100050000D1201C01201C0754000753E00754100CF
:10006000753C007539709131309008E540B4000F4F
:10007000020068E5402480F54012067302006830F3
:100080009131309231309331309431309534309613
:100090003730973A20A2D1753F5485393A12067607
:1000A000C2A130A2FDD2A1853A39753F521206761F
:1000B0000200680200D40200680200681201CD024A
:1000C00000681201F00200681201FD0200681202CD
:1000D0000D020068753C8075410012041D753B02DD
:1000E00012030D20911530925230935530945830B0
:1000F000955B30965E3097610200E312041D753BFC
:100100000312030D30905830915B30925B30935E58
:1001100030946130956430966730976A20A2E57517
:100120003F5485393A120676C2A130A2FDD2A1858C
:100130003A39753F5212067602010412021D02017D
:100140000412023102010412024502010412025992
:1001500002010412026D0201041202810201041262
:1001600001CD02010402018C120295020104120267
:10017000A90201041202BD0201041202D10201040B
:100180001202E50201041202F9020104753C001298
:1001900006761201C0020068780079007A08D8FE5D
:1001A000D9FCDAFA2278007900D8FED9FC227B9BB0
:1001B000DBFE227C007A007F01DCFEDAFCDFFA2223
:1001C000780079007A04D8FED9FCDAFA22E54124D5
:1001D00080F541B4800DE5399430F5391206761278
:1001E00001C022E5392430F5391206761201C02209
:1001F000E53E2480F53E1206761201C0221539E54F
:1002000039B4FF037539A012067631A5220539E508
:1002100039B4A1F375390012067631A52290000099
:10022000E53E12045DE53912045D753D3112067636
:1002300022900010E53E12045DE53912045D753D23
:100240003212067622900020E53E12045DE5391256
:10025000045D753D3312067622900030E53E1204AF
:100260005DE53912045D753D34120676229000403A
:10027000E53E12045DE53912045D753D35120676E2
:1002800022900050E53E12045DE53912045D753D93
:100290003612067622900000120469F53E120469B7
:1002A000F539753D3112067622900010120469F579
:1002B0003E120469F539753D32120676229000200F
:1002C000120469F53E120469F539753D331206765C
:1002D00022900030120469F53E120469F539753D2B
:1002E0003412067622900040120469F53E12046929
:1002F000F539753D3512067622900050120469F5E5
:100300003E120469F539753D3612067622C2B5747F
:100310008012038B1201AED2B5E53BB40106900604
:100320008F020375B402069006E0020375B403065B
:10033000900731020375B40406900782020375B476
:100340000506900785020375B40606900788020328
:1003500075B4070690078B020375B4080690078EE4
:10036000020375B40906900791020375B40A1B9045
:1003700007940203757400931201AEB48203020362
:100380008AA312038B740002037722A2E79287A24A
:10039000E69286A2E59285A2E49284D2B70000C2DA
:1003A000B71201AEA2E39287A2E29286A2E1928501
:1003B000A2E09284D2B70000C2B71201AE22A2E737
:1003C0009287A2E69286A2E59285A2E49284D2B7B1
:1003D0000000C2B71201AE22C2B51201B3743012CE
:1003E00003BE1201B374301203BE1201AE74301298
:1003F00003BE1201AE74201203BE1201AE742C12A1
:10040000038B740C12038B740112038B1201B374EF
:100410000612038B22C2B5740812038B22C2B57474
:100420000112038B1201B322D2A01204151201C0D3
:1004300022E540B480F2C2A01203D812041D753B1D
:100440000112030D1201C01201C07531FD75300596
:10045000C2B3C2B27F64B14EDFFCB12C224396100E
:10046000F01201B3A363961022E0A32212041DD25E
:10047000B5744612038B744D12038B742012038BD8
:10048000E541B4801E744E12038B746112038B74A9
:100490006812038B746C12038B746512038B746483
:1004A00012038BE53CB48013C2B5748D12038BD25A
:1004B000B5744D12038BE53D12038BC2B574C012A7
:1004C000038BD2B5E53F12038B745812038BE53EC4
:1004D000B48008742D12038B0204E0742012038B85
:1004E000742012038B743112038B743412038BE566
:1004F00038243012038B742C12038BE5372430120E
:10050000038BE536243012038BE535243012038B40
:10051000E534243012038B742012038B744D1203C4
:100520008B744812038B747A12038B22C2B4C2B24A
:10053000C2B3D2B3B14EE531B143E530B143C2B33A
:10054000B14E227808330092B2B14ED8F822D2B41C
:100550007D05DDFEC2B42275312974A82539F53038
:10056000E5313400F53122E53975F07DA42440F5FC
:1005700032E5F0349CF533B1F7AE33AF327A277BF6
:1005800010D1088F38B1F7AF387C277D10D15FE5E7
:1005900032C39FF532E5339EF533B1F7AE33AF3258
:1005A0007A037BE8D1088F37B1F7AF377C037DE85A
:1005B000D15FE532C39FF532E5339EF533B1F7AE37
:1005C00033AF327B64D1088F36B1F7AF367D64D15B
:1005D0005FE532C39FF532E5339EF533B1F7AE33B5
:1005E000AF327B0AD1088F35B1F7AF357D0AD15FC5
:1005F000E532C39FF53422780079007A007B007CD5
:10060000007D007E007F0022BA002CEC8BF084CFAE
:10061000CECDFCE5F0CBF97818EF2FFFEE33FEEDF1
:1006200033FDEC33FCEB33FB4003994004EB99FBC7
:100630000FD8E6E4F9FA227818EF2FFFEE33FEED3B
:1006400033FDEC33FCC933C940059BE99A4007EC04
:100650009BFCE99AF90FD8E1E4C9FAE4CCFB22EF5C
:10066000F88DF0A4FFEDC5F0CEA42EFEEC88F0A42A
:100670002EFE22120431E53FB4540BE53EB4800651
:10068000E5399430F539B167916CB157B12C2254EA
:1006900072616E736365697665722020326D202009
:1006A000202020202020202020202020202020204A
:1006B0002020202020202075726F62696C204F4B13
:1006C000325A47523A2D2920202020202020202055
:1006D00020202020202020202020202020202082B8
:1006E000556C6F7A20646F2070616D65746920208D
:1006F00020202020202020202020202020202020FA
:1007000020202020202020202020203120617A203D
:1007100036202020202020202020202020202020C3
:1007200020202020202020202020202020202020C9
:1007300082566F6C206369736C6F2070616D657495
:100740006920202020202020202020202020202060
:100750002020202020202020202020203120617AED
:100760002036202020202020202020202020202073
:100770002020202020202020202020202020202079
:10078000208220208220208220208220208220207F
:07079000822020822020825C
:00000001FF
